:020000040000FA
:060000000A3002303A282C
:08000800A000030EA100831209
:1000100005191028831601178312B23081002B288E
:1000200083160113831203140B190310A80DA90DD5
:10003000AA0DAB0DAC0DAC16FF302C02031D2B2806
:10004000FA302B02031D2B2831152A08AF0029088E
:10005000AE002808AD008B100B11210E8300A00EFE
:04006000200E090065
:0C007400203084008001840A6030040207
:10008000031C3C281230B0005F218316FF23900030
:10009000831283160C308505870183128501870141
:1000A000073099000030831691009F008312C830FA
:1000B00083168100831231309000003083168C004B
:1000C000831210308B00C42181018E018F010B112E
:1000D0008B100B108C018B177B2031197E20B30BFA
:1000E0007928031085190314B90DF030390203196A
:1000F000E820C5216C28640032100800311101305D
:10010000B7008B132030370783169B001C141A0886
:100110008312A4001030370783169B001C141A08A2
:100120008312A300A6000230A6060030370783160C
:100130009B001C141A088312A200A7000130A70616
:100140008B17321CA92822090339A200A309A4098C
:10015000A50924082F02031DE22823082E02031DEF
:10016000C32822082D02031DE22801303702031D97
:10017000BC283D143E14762102303702031DC328EB
:10018000BD143E14822126082E02031DDA282708FA
:100190002D02031DE22801303702031DD2283D1035
:1001A0003E148E2102303702031DD928BD103E14A3
:1001B0009A21E2285F08AB3C0319E2282E1AE228B4
:1001C000E128A621B70A0330370203180800812866
:1001D0000130B600B300B400B500B7008501870157
:1001E000B113B6217B20B30B112903108519031419
:1001F000B90DF030390203193829B41F8501B41F35
:100200008701B40B1129B50B11290230B50001305B
:1002100037020319AC21023037020319B121FA3039
:10022000B400311DF2283111321C1B292D0903396C
:10023000AD00AE09AF092F1CF2288E018F010C1CF6
:10024000F2280C102E1EF2288B1320303707BB002B
:100250002F08BA004C2110303707BB002E08BA0017
:100260004C2100303707BB002D08BA004C218B17FA
:10027000BD2185018701B70AB60103303702031C8F
:10028000F228C42108003E1C08003E101030BB00BC
:100290003D08BA004C2108008B133A0883161C1540
:1002A0009A003B089B0055309D00AA309D009C148D
:1002B00064009C1858291C1183128B1708008316A0
:1002C00000309B001C141A088312DF0083162030B4
:1002D0009B001C141A088312C1000130C11BC1000D
:1002E000C1080319C1004108C000080083160510A9
:1002F000851083120510851440084107D0000F08AF
:10030000D100080083160512851283120512851686
:1003100040084107D2000F08D300080083160510DB
:10032000851083128510051440084107D0000F087E
:10033000D100080083160512851283128512051656
:1003400040084107D2000F08D300080085013F3064
:100350008316850083120800380903398500B80028
:100360000800380930398500B80008003C30831691
:1003700085008312B801B81408000F308316850079
:100380008312B801B8160800080050084002031D87
:10039000D32951080F02031CD32905108510831699
:1003A00005148514831252084002031DE1295308E5
:1003B0000F02031CE1290512851283160516851606
:0C03C00083120C1C08000C10C00A08007E
:084000000C00030005000100A3
:02400E00CC01E3
:10420000010078007A007C007E007B0079007F004E
:104210007D007A0078007E007C00FF00FF00FF0038
:104220000000F200F600FA00FE00F200F600FA00CC
:10423000FE00F200F600FA00FE00FF00FF00FF00A3
:10424000010005000500050005000900090009003E
:1042500009000D000D000D000D00FF00FF00FF0024
:10426000FF00FF00FF00FF00FF00FF00FF00FF0056
:10427000FF00FF00FF00FF00FF00FF00FF00FF0046
:10428000FF00FF00FF00FF00FF00FF00FF00FF0036
:10429000FF00FF00FF00FF00FF00FF00FF00FF0026
:1042A000FF00FF00FF00FF00FF00FF00FF00FF0016
:1042B000FF00FF00FF00FF00FF00FF00FF00FF0006
:1042C000FF00FF00FF00FF00FF00FF00FF00FF00F6
:1042D000FF00FF00FF00FF00FF00FF00FF00FF00E6
:1042E000FF00FF00FF00FF00FF00FF00FF00FF00D6
:1042F000FF00FF00FF00FF00FF00FF00FF00DD00E8
:00000001FF
